:1000000000308A00D92D00000B138B138B1B0528A1
:10001000DF2D52308400000803191D280130A10093
:10002000A001A00B1128A10B10284A30A000A00BA2
:10003000172800000000800B0E2800343330CC005D
:100040003230CD002830CE000630CF000C30D0004A
:100050000130D100F0306500003066000612053036
:10006000D2000920CA014A08053C031C52284C3022
:100070004A0784000008CB0086110530D200092011
:10008000CB0E4B08850006160530D200092006125B
:10009000CB0E4B08850006160530D200092006124B
:1000A000CA0A3328E02D003049180130FE3E0318FB
:1000B0007028023E71284430C3006530C40073309C
:1000C000C5002030C600C70070284C30C30069301E
:1000D000C4006730C5004130C6004C30C7007028EE
:1000E00000340A108A100A1182075B286528423002
:1000F000A000A00B7928000000347720861177201B
:10010000CB0E4B0885007720061677200612CB0E03
:100110004B088500772006167720061200347720DA
:1001200086157720CC0E4C088500772006167720A0
:100130000612CC0E4C088500772006167720061292
:1001400000348030CB007D205030CC008F206130D7
:10015000CC008F207230CC008F206130CC008F20FB
:100160002030CC008F206130CC008F206A30CC0052
:100170008F207530CC008F207330CC008F207430EE
:10018000CC008F206130CC008F207230CC008F20CB
:100190002030CC008F206130CC008F202030CC006C
:1001A0008F202030CC008F20C030CB007D206830E5
:1001B000CC008F206F30CC008F207230CC008F208D
:1001C0006130CC008F202030CC008F206530CC00F7
:1001D0008F202030CC008F206130CC008F20203049
:1001E000CC008F206430CC008F206130CC008F2079
:1001F0007430CC008F206130CC008F202030CC00B8
:100200008F202030CC008F202030CC008F20083071
:10021000CA00FA30D2000920CA0B09298030CB006D
:100220007D205030CC008F207230CC008F20653084
:10023000CC008F207330CC008F207330CC008F2007
:100240006930CC008F206F30CC008F206E30CC0016
:100250008F206530CC008F202030CC008F20533091
:10026000CC008F204530CC008F205430CC008F2024
:100270002030CC008F206530CC008F202030CC0087
:100280008F20C030CB007D206330CC008F206F30BA
:10029000CC008F206E30CC008F206630CC008F20B9
:1002A0006930CC008F207230CC008F206D30CC00B4
:1002B0008F206530CC008F202030CC008F2065301F
:1002C000CC008F206D30CC008F202030CC008F20D0
:1002D0004D30CC008F204F30CC008F204430CC00EC
:1002E0008F204530CC008F200830CA00FA30D20071
:1002F0000920CA0B7629EE2D01302802F93E031899
:10030000B429073EB5295330AC006530AD006730E5
:10031000AE00B4295430AC006530AD007230AE0090
:10032000B4295130AC007530AD006130AE00B42955
:100330005130AC007530AD006930AE00B429533097
:10034000AC006530AD007830AE00B4295330AC005D
:100350006130AD006230AE00B4294430AC006F3083
:10036000AD006D30AE00B42900340A148A100A11B1
:10037000820783298A29912998299F29A629AD29AD
:100380008030CB007D2030303307CB00CC008F2075
:1003900030303A07CB00CC008F202F30CC008F209C
:1003A00030303407CB00CC008F2030303B07CB00FF
:1003B000CC008F202F30CC008F203230CC008F200B
:1003C0003030CC008F2030303507CB00CC008F2070
:1003D00030303C07CB00CC008F202030CC008F2069
:1003E0002030CC008F202030CC008F202C08CC0077
:1003F0008F202D08CC008F202E08CC008F20C030FD
:10040000CB007D2030303107CB00CC008F20303046
:100410003807CB00CC008F203A30CC008F20303012
:100420003007CB00CC008F2030303707CB00CC001A
:100430008F203A30CC008F2030302F07CB00CC00FB
:100440008F2030303607CB00CC008F202030CC00FE
:100450008F202030CC008F202030CC008F20203007
:10046000CC008F202030CC008F202030CC008F207B
:100470004608CC008F204708CC008F200034A00114
:10048000A101520803105318A007A00CA10CD31807
:10049000A007A00CA10C5319A007A00CA10CD31904
:1004A000A007A00CA10C531AA007A00CA10CD31AF2
:1004B000A007A00CA10C531BA007A00CA10CD31BE0
:1004C000A007A00CA10C00340830A100000000001F
:1004D00006118316061100008312CC0D8610031C32
:1004E000742A8316861483120318792A83168610B9
:1004F0008312831606158312061D7C2AA10B662A19
:10050000000006118316061100008614000000008A
:1005100006158312061D8A2AA101000086182114DF
:100520000611831606118312861083168610831215
:100530000034B601AF01B701B001B801B10101301B
:10054000B900B201BA00B301BB00B4010730BC006E
:10055000B5013908A8007C21C021A5018316061722
:100560008312061FCE2A831686168312861ACD2A78
:10057000B80A3808093C0318BF2AB801B10A310883
:10058000023C031DC92A3808043C031DC92AB101D5
:10059000B801C0219630D2000920AE2A3108D2001D
:1005A0000A30D3003F2238082107A7008316061718
:1005B0008312061FD62AC021831606178312061F30
:1005C000F72A831686168312861AF62AB70A370880
:1005D000093C0318ED2AB701B00A3008053C03189E
:1005E000F22AB001C0219630D2000920DC2A30085E
:1005F000D2000A30D3003F2237082107A600831615
:1006000006178312061FFF2AC021831606178312BE
:10061000061F262B831686168312861A252BBA0AE6
:100620003A08093C0318162BBA01B30A3308033CF5
:10063000031D212B3A08023C031D212BB30101307D
:10064000BA00C0219630D2000920052B3308D20011
:100650000A30D3003F223A082107A9008316061763
:100660008312061F2E2BC021831606178312061F26
:10067000532B831686168312861A522BBB0A3B080D
:10068000093C0318452BBB01B40A340B4E2B3B0825
:10069000033C031D4E2BB4010130BB00C02196303A
:1006A000D2000920342B3408D2000A30D3003F2274
:1006B0003B082107AA00831606178312061F5B2B2F
:1006C000C021831606178312061F802B83168616F9
:1006D0008312861A7F2BBC0A3C08093C0318722B34
:1006E000BC01B50A350B7B2B3C08063C031D7B2B5C
:1006F000B5010730BC00C0219630D2000920612B23
:100700003508D2000A30D3003F223C082107AB0055
:10071000831606178312061F882B3908A8007C2130
:10072000C021831606178312061FAA2B831686166E
:100730008312861AA92BB90A3908073C0318A22B81
:100740000130B9003908A8007C21C0219630D200C0
:100750000920912BCA014A08063C031CD02B2530E6
:100760004A07CB0025304A0784000008CC00CD00A2
:100770004D08CE00CF014E08093C0318C42B0A30A7
:10078000CE021030CF07C72B4E08CF07C82BBB2B8C
:100790004F08A1004B08840021088000CA0AAB2B37
:1007A0001430D200092083168614000006150000BC
:1007B000831286108316861000008312061183169A
:1007C0000611D0308312CC006422CC016422CA010D
:1007D0004A08063C031CF52B25304A078400000814
:1007E000CB00CC006422CA0AE82B1030CC00642273
:1007F00083168610000006158312061DFD2B0000CF
:100800000000000000008316861400008312EF2D04
:100810008030CB007D204130CC008F206A30CC006E
:100820008F207530CC008F207330CC008F20743037
:10083000CC008F206130CC008F207230CC008F2014
:100840002030CC008F206130CC008F206C30CC0069
:100850008F206130CC008F207230CC008F206D3023
:10086000CC008F206530CC008F202030CC008F2032
:100870002030CC008F20C030CB007D2030304007AE
:10088000CA00CC008F2030304207CA00CC008F2035
:100890003A30CC008F2030303F07CA00CC008F2088
:1008A00030304107CA00CC008F202030CC008F2090
:1008B0002030CC008F202030CC008F202030CC0086
:1008C0008F202030CC008F204308CC008F2044089C
:1008D000CC008F204508CC008F202030CC008F200A
:1008E0002030CC008F202030CC008F2000345320CB
:1008F0000824831606178312061FA12C831686165A
:100900008312861A982CC20A4208093C03188A2CC2
:10091000C201C00A4008023C031D942C4208043C5A
:10092000031D942CC001C20108249630D200092076
:100930004008D2000A30D3003F2242082107BE00FF
:10094000792C831606178312061FA12C08249630D3
:10095000D2000920831606178312061FCD2C83169A
:1009600086168312861AC42CC10A4108093C031852
:10097000BB2CC101BF0A3F08053C0318C02CBF01B6
:1009800008249630D20009203F08D2000A30D30054
:100990003F2241082107BD00AA2C831606178312A7
:1009A000061FCD2C0824831606178312061FE52C7C
:1009B000831686168312861AE42C0130C90653204A
:1009C00008249630D2000920D32CF52D0830CC0015
:1009D0002008CD0083168614000006158312061D1C
:1009E000EF2C86180314861C0310A10D000083163B
:1009F000061183120611CC0BEA2C83168614000014
:100A0000831286104D080319082D83168610831251
:100A10000000831606158312061D0C2D000006111A
:100A20008316061100008312861083168610831227
:100A30000034831686140000061500008312861009
:100A40008316861000008312061183160611D0301B
:100A50008312CC006422CC01642283168614000029
:100A6000061500008312861083168610000083127C
:100A7000061183160611D1308312CC006422013096
:100A8000A000E62421087F39A5000130A000E6245B
:100A900021087F39A6000130A000E62421083F3953
:100AA000A7000130A000E62421080739A800013082
:100AB000A000E62421083F39A9000130A000E62467
:100AC00021081F39AA00A001E6242108AB008316E3
:100AD0008610000006158312061D6C2D0000000014
:100AE0000000000083168614000083127C21CA01D6
:100AF0004A08063C031CB92D25304A07CB00253097
:100B00004A0784000008CC00CD004D08CF000F300C
:100B1000CF054F08D0003630480784004F088000CA
:100B20004D08CF00CE014E08033C031C9B2D031043
:100B3000CF0CCE0A932D2F30480784004F08800039
:100B40004F08D2000A30D3003F222108CF00D10045
:100B500050085107CF00C80A4808063C0318B12DB9
:100B6000C8014F08A1004B08840021088000CA0A70
:100B7000782DF62D4911831686168312861EC52DF3
:100B8000831606178312061BC62DC910CA014A0810
:100B9000633C031CD52D06140130D2000920061039
:100BA0000130D2000920CA0AC72DC830D20009205E
:100BB000142E84011F30830507309F0004281E284F
:100BC000C801BF01C101C001C2014910C9104915C6
:100BD00053200610C830D2000920A128992A831674
:100BE00086178312861BF52D772C192D5320C021D3
:100BF000003049190130013C031D0D2E26083D022D
:100C0000031D0D2E27083E02031D0D2E003049182E
:100C10000130013C031D0D2EC9140030C9180130EC
:100C2000013C031D142EBA2D26083D02031D1C2E67
:0E0C300027083E0203191D2E4915EF2D630003
:02400E00183F59
:00000001FF
